:100000007B2B820700340034013401340234023483
:100010000334033404340534063407340834093413
:100020000A340B340C340E341034123414340F30C0
:10003000831201058207000000000000000000009C
:1000400000000000000000000000000000000000B0
:100050000000000045088500E2308100410884006E
:100060000508C200C30A0008C400840A0008C500CD
:10007000840A4C30841E0408C1004408850008002E
:10008000A2011430220203184B284C3022078400AE
:100090008001A20A41284C30C100C501FC3081001A
:1000A0001728FF2383169000083085008312101054
:1000B0000C1008308316810083121016901610144D
:1000C00019159914191483169F01831285010800CC
:1000D000A3000E08B60033083602031CB40A360823
:1000E000B30023083607B5000E083506031D742833
:1000F0000800A200B40164303402031887282230BB
:100100008500220868208501220868207B280800D5
:10011000B40164303402031890280A30682089281A
:100120000800B301B4018E0157307920673079207F
:1001300088208820882067307920613079205730E6
:10014000792033307920882033307920882041305D
:100150007920882088208828A30083128C13220805
:1001600083169B0023089A001C1555309D00AA3069
:100170009D009C141C1183128C1FBB2883128C13AE
:1001800083120800A200220883169B001C141A0880
:10019000A3008312230808000030C220B9003908E8
:1001A0002A3A031DD7280130C220B900DB28A2015A
:1001B0002A30AC20B90108001C30BA001C30BB004A
:1001C0001C30BC001C30BD002730BE002730BF00F3
:1001D0002730C0000800BA1B17281720AD080319E4
:1001E000F3281C30BA00BA031720BA1F00290130C7
:1001F000A2003908AC2017200A30AB000A30AC004E
:10020000BB1B1E291720AC1F0929F7302C02031C29
:100210000B291C30BB001720AB1B12290A302B0204
:1002200003181B291720AB1F1929F7302B02031CB9
:100230001B291C30BB001720BB0330291720AB1B28
:1002400028290A302B02031C2829391417202929B0
:10025000391017201C30BB000A30AB000A30AC004C
:100260001720BC1B4F291720AC1B3A2909302C0240
:1002700003183C291C30BC001720AB1B4329093054
:100280002B0203184C291720AB1F4A29F6302B02EA
:10029000031C4C291C30BC001720BC035F2917200D
:1002A000AB1B592909302B02031C5929B9141720FB
:1002B0005A29B91017201C30BC00AB01AC01172023
:1002C000BD1B6E291720AD1B692914302D020318A0
:1002D0006B291C30BD001720BD037B2917202B087C
:1002E000BE072C08BF072E08C0071C30BD000A300F
:1002F000AB000A30AC001720AD0117281720C6014B
:10030000C301172008300505290603199D29C31FBD
:100310008129C301172008300505290603199D29E5
:10032000C31F8A29C30117200830050529060319B0
:100330009D29C31F932917200134C30117200830BA
:10034000420529060319C60A172000341720A30105
:10035000043023020318E62917201A30C30217209D
:10036000083005052906031DB929C31BAF2917202D
:10037000013417201A304307B7001720B71BC329D1
:1003800002303702031C0134E530C3071720083060
:10039000050529060319D029C31BC62917200134D6
:1003A000172034304307B70017202B302307840071
:1003B000370880000230C3001720B71BE22919302C
:1003C0003702031C01341720A30AA82917202A0882
:1003D000033A031DF4292D08B70017202E08AD009D
:1003E0003708AE001720003417202A0B002A2C08EB
:1003F000B70017202D08AC003708AD0017200034D7
:100400001720AA08031D122A2B08B70017202C0852
:10041000AB003708AC002C08B70017202D08AC0043
:100420003708AD001720003417202F082B07AF0026
:100430000310AF0C2F08AB00172030082C07B000BA
:100440000310B00C3008AC00172031082D07B100A4
:100450000310B10C3108AD00172032082E07B2008E
:100460000310B20C3208AE0017203E08AB023F0862
:10047000AC021E30AD024008AE021720AD1BAD012C
:10048000EB201720391C4A2A2B08B7002C08AB0296
:100490003708AC071720AB1F522AAB09AB0A013053
:1004A000B300542A0230B3001720AC1F5C2AAC09F9
:1004B000AC0A1030B4005E2A2030B4001720AE1F02
:1004C000652AAE09AE0AB601662AB60117202B08C6
:1004D000AB072C08AC072E08AE071720AB1B762AFB
:1004E00015302B02031C762A1430AB001720AC1BEE
:1004F0007F2A15302C02031C7F2A1430AC001720F1
:10050000AD1B882A15302D02031C882A1430AD003B
:100510001720AE1B912A15302E02031C912A14308D
:10052000AE001720B91C172817202B080120AB009C
:1005300017202C080120AC0017202E080120AE0047
:100540001728A501A601A701A8011720A3011430AF
:100550002302031817281720A2012B08A502A51FA4
:10056000B62A17201430A5073308A20717202C0835
:10057000A602A61FC02A17201430A6073408A20717
:1005800017202D08A702A71FCA2A17201430A70773
:100590003508A20717202E08A802A81FD42A172062
:1005A0001430A8073608A20717204C302307840010
:1005B000220880001720A30AA72AAD01B801043041
:1005C000B500080017200630C70080300F07C800AC
:1005D0000800172048080F028039031D172817202C
:1005E0008030C807C708031D1E2B17200630C70020
:1005F0000230AB000130B3001720391C022B02304F
:10060000AC00032BAC0117201030B4003808AD004B
:100610000230AE00B6011720A12217200314AD1F2F
:1006200003102D0CB7002D08B70717200314B71FB0
:100630000310370CAD0017202D08B800C70317288A
:10064000172006300F07CA0002300F07C900172015
:1006500049080F0280390319442B1720083005057B
:100660002906031D422B172002300F07C900290855
:10067000083CA90017204A080F028039031D422BAD
:10068000172001341720282B1720003417200230A0
:10069000AA0017202023003A0319502B17204A2BB9
:1006A0007E21003A031D492B1720A621003A031989
:1006B0005B2B1720492BB3011720A2010430220223
:1006C0000318172817202B30220784000008B700D2
:1006D00017202730B702B71F6F2BB709B70A1720AB
:1006E00033083702031C782B3708B3002208AA000E
:1006F0001720A20A5E2B51209120CC20DD22A001E0
:10070000DC20A901A1010430210203188E2B2F3017
:100710002107840027308000A10A832B4020462334
:10072000A0080319E22217200430A0001720172088
:10073000A008031DE92217202023003A031DB92B2E
:1007400017207E21003A031DB92B1720A621003A5D
:10075000031DB92B172014221720A0080319B32B4F
:10076000A0031720972B1720A12217202D08B800CF
:06077000972B1720902BCF
:0207FE000934BC
:044200002A00000090
:02400E00843FED
:00000001FF
